:020000040800F2
:100000006009002045010008491600085513000842
:1000100045160008690200080332000800000000CD
:10002000000000000000000000000000B5280008EB
:10003000ED0F000800000000B5220008152B000895
:100040005F0100085F0100085F0100085F01000810
:100050005F0100085F0100085F0100085F01000800
:100060005F0100085F0100085F0100085F010008F0
:100070005F0100085F0100085F0100085F010008E0
:100080005F0100085F0100085F0100085F010008D0
:100090005F0100085F0100085F0100085F010008C0
:1000A0005F0100085F0100085F0100085F010008B0
:1000B0005F010008792B00085F0100085F0100085C
:1000C0005F0100085F0100085F0100085F01000890
:1000D0005F010008592D0008B52D0008992E000871
:1000E0005F0100085F0100085F0100085F01000870
:1000F0005F0100085F0100085F0100085F01000860
:100100005F0100085F0100085F0100085F0100084F
:100110005F0100085F0100085F0100085F0100083F
:100120005F0100085F0100085F0100085F0100082F
:10013000DFF80CD000F03CF800480047DD34000840
:10014000600900200648804706480047FEE7FEE7B2
:10015000FEE7FEE7FEE7FEE7FEE7FEE7FEE7FEE777
:10016000192B00083101000840EA01039B0703D066
:1001700009E008C9121F08C0042AFAD203E011F8E6
:10018000013B00F8013B521EF9D27047D2B201E0A8
:1001900000F8012B491EFBD270470022F6E710B58C
:1001A00013460A4604461946FFF7F0FF204610BDE5
:1001B000064C074D06E0E06840F0010394E80700B4
:1001C00098471034AC42F6D3FFF7B6FFF43C000872
:1001D000143D000808B54FF48070ADF80000102001
:1001E0008DF8030003208DF8020069461C4800F0DA
:1001F000FAFF4FF48070ADF800006946194800F02E
:10020000F2FF1020ADF800006946164800F0EBFF41
:100210002020ADF800006946124800F0E4FF4FF4DA
:100220008040ADF8000069460E4800F0DCFF4FF456
:1002300080710B4801F062F84FF48071094801F0B9
:100240005DF81021074801F059F82021054801F018
:1002500055F84FF48041034801F050F808BD000004
:10026000000801400010014000BFFEE710B5024643
:100270000B460020002104E0545C0444E0B24C1C16
:10028000E1B29942F8DBC443E0B2441CE0B210BDD5
:10029000FEB5002000900190029001F0A3F94B48B8
:1002A00000780A281DD14A4800784A4909788842CE
:1002B00017D14748407847494978884211D1444886
:1002C000007A4449097A88420BD14148407A414931
:1002D000497A884205D14048008840F400403E49B0
:1002E00008803D48008800F4004000286CD00120C0
:1002F00003F05EF800203949087048708870C870B3
:1003000008713749087048708870C870087135499D
:10031000087048708870C870087133490870487058
:100320008870C870087101F05DF900202C490870D0
:100330002748007948702648407988702448807999
:10034000C8702348C07908710020284908702448E3
:10035000407848702248807888702148C078C870FA
:100360001F4800790871012001F036FB1C484078D5
:1003700007061B48807804041948C078050238191C
:1003800028441749097946180A226946304600F080
:10039000F3FF022003F074FA062315A201210220C4
:1003A00003F032FB0A236A460721022003F02CFBEC
:1003B00001201149087001F015F901F013F900202E
:1003C0000249087004490880FEBD000009000020B1
:1003D000D80100200C0000200A0000202C00002082
:1003E0001600002034000020390000201B000020EF
:1003F00031332E35363A00004100002010B588B068
:100400007F480078012838D100207D490870FC2001
:100410007C490870112048707B48007888707A48C1
:100420004078C8707848807808717748C0784871FB
:1004300075480079887107217248FFF717FF7149E5
:10044000C871002071490860FF22E121012001F0FC
:100450007FFE08236B4AA821012001F03BFE01200A
:1004600001F0BAFA01206A49C1F8A401694908708B
:1004700000206949088001F0B5F86748008840F617
:10048000B83188427BDC01F0ADF860488438006800
:10049000002857D101F0A6F86946012001F0F8FDC7
:1004A0000446204602F054FA5CA002F05BFA04F025
:1004B00040004028EDD100208DF80A000721684651
:1004C00000F095FD55A002F04DFA9DF801004E494F
:1004D0000978884254D19DF802004B4949788842F6
:1004E0004ED19DF8030048498978884248D19DF84B
:1004F00004004549C978884242D19DF80500424927
:10050000097988423CD14348007801281BD14148F1
:100510000078401C3F49087012203A494870072172
:100520003848FFF7A3FE3749C871002037490860F3
:100530000823344AA821012001F0CCFD01203449D0
:10054000C1F8A40158E00020324908700E21344857
:1005500000F04DFD31A002F005FA3248017801208B
:1005600001F094FA10202E4948700E212C4802F018
:10057000E3F92DA002F0F6F9012008B010BD16E055
:1005800000202249086011201E49487007211D489B
:10059000FFF76CFE1B49C87108230A46A8210120F9
:1005A00001F098FD01201A49C1F8A40124E00020BF
:1005B0001549087048708870C87008711B49087028
:1005C00048708870C8700871194908704870887040
:1005D000C87008711749087048708870C870087131
:1005E00030200F4948700E210D4802F0A5F912A0E5
:1005F00002F0B8F90120C0E700F0F4FF0020BCE7EA
:100600003E000020420000202C000020A481214256
:100610000080214282000020200000200A0000000B
:10062000CC0300202A0000204F4B0A003900002094
:100630001B00002016000020333030300A0000007C
:1006400010B588B03C48008840F2DC51884268DA36
:100650003A480068002861D100F0C4FF69460120D3
:1006600001F016FD044604F04000402856D1002059
:100670008DF80A000721684600F0B9FC30A002F0AE
:1006800071F99DF8010078B99DF8020060B99DF8F4
:10069000030048B900202B49087048708870C87062
:1006A0000871012008B010BD2748007807280FD135
:1006B0000020244908709DF8000048709DF8010052
:1006C00088709DF80200C8709DF80300087123E04F
:1006D0001D480078082810D19DF8010019490870BC
:1006E0009DF8020048709DF8030088709DF8040092
:1006F000C8709DF8050008710EE0002011490870CF
:100700009DF8010048709DF8020088709DF8030074
:10071000C8709DF8040008710120C3E700F062FF73
:1007200008E000200749087048708870C870087198
:100730000120B7E70020B5E73200002020812142E8
:100740000A000000390000202A0000203EB50020E9
:100750000090019002904748007800287ED04648DB
:100760000178012001F092F900204449088004E05A
:10077000FFF766FF044604B100E0F9E700BF002080
:100780003C4908703E48407800063D49897840EA77
:1007900001403B49C97840EA01203949097940EADA
:1007A00001050A226946284600F0E6FD032003F011
:1007B00067F8032333A20121184603F025F90A2321
:1007C0006A460421032003F01FF916212E4802F087
:1007D000B3F8322002F0ECFD16212B4800F007FCA4
:1007E0002AA002F0BFF82A480078254909788842F3
:1007F00021D1274840782249497888421BD1244892
:1008000080781F498978884215D12148C0781C49D1
:10081000C97888420FD11E48007919490979884260
:1008200009D1042003F02CF802231AA2042108465F
:1008300003F0EAF808E0042003F022F8022316A2ED
:100840000421084603F0E0F800200D4908704870C4
:100850008870C87008710E49087000E009E048709F
:100860008870C87008710D49087048708870C87029
:1008700008713EBD410000202A0000203200002007
:100880003900002049443A00680300200A000000B3
:100890001B0000204F4B00004E47000016000020B8
:1008A0003EB5002000900190029000F09BFEFE48B3
:1008B0000078082829D1FD480078752825D1FB4803
:1008C0004078702821D1F948807864281DD1F748F4
:1008D000C078612819D1F5480079742815D1F348FA
:1008E0004079652811D10020EF49087000BFF04819
:1008F000006800F4E060EF490843001DEC4908601F
:10090000BFF3408F00BF00BFFEE7E84800787528BE
:1009100007D0E6480078FA2803D00020E2490870A2
:100920003EBDE14800780E2800DAF9E7DE4800789D
:10093000401EDE49085CFB2800D0F1E7DB48807AE6
:10094000A02804D1D8480078152800D0E8E7D64878
:1009500000780E281ED1D5480078FA2814D1D34843
:10096000407BFB2810D1D448008840F40040D24995
:1009700008800020CC4908700E21CC4800F037FBDD
:10098000CEA001F0EFFF4AE00020C7490870CA4935
:10099000088044E0C448007815281ED1C348007878
:1009A000FA2814D1C148007DFB2810D1C248008824
:1009B00040F40040C04908800020BB490870152160
:1009C000BA4800F014FBBDA001F0CCFF27E00020E6
:1009D000B5490870B849088021E0B348007811286B
:1009E0001DD1B2480078FA2814D1B048007CFB2809
:1009F00010D1B148008840F40040AF490880002081
:100A0000A94908701121A94800F0F1FAABA001F042
:100A1000A9FF04E00020A4490870A7490880A6485F
:100A2000008800F40040002871D000F0DBFD9F48F2
:100A30008079A34988719D48C179A148C1719B48BB
:100A4000017A9F4801729948417A9D4841729748BE
:100A5000807A9B498872084680799A4988719848BB
:100A6000C1799848C1719648017A964801729448B4
:100A7000417A944841729248807A94284CD018DC8C
:100A8000732834D00CDC252825D004DC21281AD08A
:100A900022287DD11BE0262821D07128F9D122E01F
:100AA000742828D075282AD078282CD08228F0D114
:100AB0002EE0A03809286BD2DFE800F0329CA0F5C8
:100AC000F4F3F2F1F00000207D498872CBE10020C0
:100AD0007B498872C7E1002079498872C3E1002010
:100AE00077498872BFE1002075498872BBE1002018
:100AF00073498872B7E1002071498872B3E1002020
:100B00006F498872AFE100206D498872ABE1AEE1B8
:100B100000206B498872A6E1002069498872A2E131
:100B20000020614908706648807967498871644887
:100B3000C1796548C1716248017A634801726048B1
:100B4000417A614841725E48807A5F4988725748AD
:100B5000407B5B4948735548817B594881735348B2
:100B6000C17B5748C1735148017C554801744F48B7
:100B7000417C534841744D48407B544908704B4870
:100B8000807B48704948C07B88704848007C00E002
:100B900068E1C8704548407C087101204C490870E4
:100BA00000204C490880012000F016FF4AA001F007
:100BB000D9FE04E0FFF722FC044604B100E0F9E7A7
:100BC00000BF45A001F0CEFE0020454908704870E6
:100BD0008870C87008714349087048708870C87080
:100BE00008714149087048708870C87008713449AC
:100BF000887238E100203249887234E139484078FF
:100C000048B93848807830B93648C07818B935487E
:100C1000007900B927E1002023490870284880792D
:100C2000324988712648C1793048C1712448017A17
:100C30002E4801722248417A2C4841722048807A1D
:100C40002A4988720120C872062008730020487360
:100C50002448017825488173224841782348C1738C
:100C600020488178214801741E48C1781F4841748A
:100C70001C4801791D488174162101F05DFE322067
:100C800002F096FB1621194800F0B1F90BA001F013
:100C900069FE002013490870487029E099E0DDE002
:100CA000D8E0D3E02BE029E0030000201001002071
:100CB0000CED00E00000FA05040000200A0000002E
:100CC00004030020A0020020CC0300202C00002000
:100CD0003E00002020000020303030300A000000AC
:100CE000390000201B0000201600002068030020AF
:100CF0008870C87008715F498872B4E0B3E0002062
:100D00005D4908705D480178012000F0BFFE0020B9
:100D10005B4908805BA001F025FE04E0FFF790FC32
:100D2000044604B100E0F9E700BF56A001F01AFE46
:100D300050488079554988714E48C1795348C171EE
:100D40004C48017A514801724A48417A4F484172F1
:100D50004848807A4D4988720120C872062008737D
:100D6000002048734A4801784848817348484178D0
:100D70004648C17346488178444801744448C17864
:100D8000424841744248017940488174162101F07B
:100D9000D3FD322002F00CFB16213C4800F027F96D
:100DA00039A001F0DFFD00203949087048708870D3
:100DB000C87008713749087048708870C870087129
:100DC0003549087048708870C87008712949887260
:100DD00049E03248407B29490870264880793049EB
:100DE00088712448C1792E48C1712248017A2C4863
:100DF00001722048417A2A4841721E48807A284967
:100E00008872012048700E21254801F095FD32209E
:100E100002F0CEFA194800782249088001F054FD0A
:100E200000201B49087048708870C8700871194903
:100E3000087048708870C870087117490870487049
:100E40008870C87008710B4988720CE0002009494D
:100E5000887208E000200749887204E000200549F4
:100E6000887200E000BF00BF00200F49088000BF6B
:100E700056E5000004030020030000202A000020A3
:100E800032000020343434340A00000068030020AB
:100E9000390000201B000020160000201001002057
:100EA000300400203805002004000020FA204A49C0
:100EB0000870102048700020887000214648C170DA
:100EC0000171417100204449887100214248C1717B
:100ED0000172417200204049C87400213E480175EA
:100EE000FB203D494875FA203C49087010204870A5
:100EF0000020887000213948C170017141710020C3
:100F00003649887100213548C17101724172002053
:100F1000324981F84B000021304880F84C10FB200A
:100F20002E4981F84D00FA202D4908701020487094
:100F30000020887000212A48C17001714171002091
:100F40002749887100212648C17101724172002031
:100F50002349C872002122480173FB2020494873AD
:100F6000FA20204908701020487000208870002165
:100F70001C48C1700171417100201A49887100211B
:100F80001848C1710172417200201649C8740021CD
:100F900014480175FB2013494875FA20124908705E
:100FA000102048700020887000210F48C170017126
:100FB000417100200C49887100210B48C1710172F8
:100FC000417200200849C872002107480173FB20C4
:100FD0000549487370470000A00200200403002068
:100FE0003004002068030020CC03002070472DE966
:100FF000F04104460E460DE02578281100F0ACF9CA
:10100000074601F0A5FC284600F0A6F9074601F0C6
:101010009FFC641C3000A6F10101CEB2ECD1BDE80A
:10102000F08100002DE9FF410E4615461F46684637
:1010300001F0E9FC9DF80000401EC0B200900428B9
:1010400001DBBDE8FF81701EC0B20646102800DB40
:10105000F7E79DF800004006000E0090F006060E2F
:1010600031469DF8000002F0FBF800201649087098
:10107000002408E015B1285D134908701348006882
:101080008047601CC4B2BC42F4DB9DF80010491CD0
:10109000C8B2314602F0E4F808E015B1285D0A490B
:1010A00008700A4800688047601CC4B27800A042FB
:1010B000F3DCAF200649096888472F2004490968F6
:1010C000884700BFBDE70000880000209000002096
:1010D0008C00002030B5044604254FF4302000F089
:1010E0006FF80546042D17D10C48006940F0020046
:1010F0000A49086108464461006940F040000861FF
:101100004FF4302000F05CF805460448006941F6D1
:10111000FD71084001490861284630BD00200240A9
:1011200004200B49C96801F0010109B101200EE05A
:101130000749C96801F0040109B1022007E0044928
:10114000C96801F0100109B1032000E004207047D4
:10115000002002400348006940F080000149086116
:10116000704700000020024070B504460D4604267A
:10117000F00200F025F80646042E11D10948006956
:1011800040F00100074908612580F00200F018F8DE
:1011900006460448006941F6FE71084001490861AD
:1011A000304670BD002002400248034948600348B1
:1011B000486070472301674500200240AB89EFCDAE
:1011C00000B502460423FFF7ABFF034603E0FFF739
:1011D000A7FF0346521E012B01D1002AF7D102B905
:1011E0000523184600BD2DE9F041024600250026E2
:1011F000002000230024002791F803C00CF00F0505
:1012000091F803C00CF0100CBCF1000F03D091F862
:1012100002C04CEA050591F800C0BCF1000F31D0C6
:10122000146800202BE04FF0010C0CFA00F3B1F829
:1012300000C00CEA03069E4220D183004FF00F0C41
:101240000CFA03F7BC4305FA03FC4CEA040491F8DA
:1012500003C0BCF1280F06D14FF0010C0CFA00FCC2
:10126000C2F814C00AE091F803C0BCF1480F05D1E0
:101270004FF0010C0CFA00FCC2F810C0401C08280A
:10128000D1D31460B1F800C0BCF1FF0F34DD546855
:1012900000202EE000F1080C4FF0010808FA0CF3D2
:1012A000B1F800C00CEA03069E4221D183004FF042
:1012B0000F0C0CFA03F7BC4305FA03FC4CEA0404D8
:1012C00091F803C0BCF1280F05D100F1080C08FA11
:1012D0000CF8C2F8148091F803C0BCF1480F07D194
:1012E00000F1080C4FF0010808FA0CF8C2F8108061
:1012F000401C0828CED35460BDE8F081416170479E
:101300000161704701460A8890B2704770B5044683
:101310000D46302C05DB392C03DCA4F1300084B2FF
:101320000EE0412C05DB5A2C03DCA4F1370084B21B
:1013300006E03A2C01D1252402E02E2C00D12424F1
:10134000034800EB041110222846FEF70DFF70BD84
:10135000933A000800BFFEE70146002001F00F02AB
:10136000092A04DC01F00F0202F1300003E001F071
:101370000F023732D0B2704730B5914BB0FBF3F368
:101380000B70904BB0FBF3F30C7804EB8404A3EBED
:1013900044034B708C4BB0FBF3F30C7804EBC405A7
:1013A00005EB0414A3EB84034C7804EB8404A3EB57
:1013B00044038B70854BB0FBF3F30C7804EB4405CE
:1013C000C5EBC414A3EBC4034C7804EBC40505EBD4
:1013D0000414A3EB84038C7804EB8404A3EB440390
:1013E000CB707B4BB0FBF3F40B7801256B43A4EB84
:1013F00003134C7804EB4405C5EBC414A3EBC403FE
:101400008C7804EBC40505EB0414A3EB8403CC78BF
:1014100004EB8404A3EB44030B7142F21073B0FBA2
:10142000F3F40B7805256B43A4EB43144B780125AB
:101430006B43A4EB03138C7804EB4405C5EBC41495
:10144000A3EBC403CC7804EBC40505EB0414A3EBB5
:1014500084030C7904EB8404A3EB44034B714FF435
:101460007A73B0FBF3F40B7801256B43A4EB831480
:101470004B7805256B43A4EB43148B7801256B4314
:10148000A4EB0313CC7804EB4405C5EBC414A3EB25
:10149000C4030C7904EBC40505EB0414A3EB84032B
:1014A0004C7904EB8404A3EB44038B716423B0FBFD
:1014B000F3F40B7801256B43A4EBC3144B786B4317
:1014C000A4EB83148B7805256B43A4EB4314CB78F2
:1014D00001256B43A4EB03130C7904EB4405C5EB26
:1014E000C414A3EBC4034C7904EBC40505EB04144A
:1014F000A3EB84038C7904EB8404A3EB4403CB714A
:101500000A23B0FBF3F40B7801256B43A4EB03240F
:101510004B786B43A4EBC3148B786B43A4EB83141D
:10152000CB7805256B43A4EB43140B7901256B4362
:10153000A4EB03134C7904EB4405C5EBC414A3EBF3
:10154000C4038C7904EBC40505EB0414A3EB8403FA
:10155000CC7904EB8404A3EB44030B720B780124D5
:101560006343A0EB43244B7801256B43A4EB032496
:101570008B786B43A4EBC314CB786B43A4EB83143D
:101580000B7905256B43A4EB43144B7901256B4381
:10159000A4EB03138C7904EB4405C5EBC414A3EB53
:1015A000C403CC7904EBC40505EB0414A3EB84035A
:1015B0000C7A04EB8404A3EB44034B7230BD0000AF
:1015C00000CA9A3B00E1F5058096980040420F0062
:1015D000A08601004CF6CC4001490860704700002D
:1015E0000030004010B500F013F810BD70B505468E
:1015F0000C4645F2555000F01FF8284600F010F850
:10160000204600F013F800F003F8FFF7E3FF70BD89
:101610004AF6AA20014908607047000000300040E7
:10162000014948607047000000300040014988606F
:10163000704700000030004001490860704700001A
:101640000030004000BFFEE7704700007CB5054653
:1016500012A103C9CDE900010821284601F002F9D1
:1016600005236A463021284600F034FD05236A46EA
:101670001021284600F09EFC002406E01DF804001E
:10168000A52800D003E0601CC4B2052CF6DB00BF27
:10169000052C01D001207CBD0020FCE7A5A5A5A557
:1016A000A500000008B501211C2000F015FE402017
:1016B000ADF8000010208DF8030003208DF8020023
:1016C00069463048FFF78FFD40212E48FFF718FE8E
:1016D0001020ADF8000069462B48FFF784FD10216B
:1016E0002948FFF70DFE0120ADF8000048208DF8D5
:1016F000030003208DF8020069462348FFF773FDBD
:101700004FF40070ADF8000010208DF803000320A6
:101710008DF8020069461B48FFF765FD4FF4007124
:101720001848FFF7EDFD4FF48050ADF80000694612
:101730001448FFF758FD4FF480511248FFF7E0FDC1
:101740004FF48070ADF8000048208DF803000320AE
:101750008DF8020069460B48FFF745FD00F0B0FF29
:1017600000F06CFF00200949086001200849C1F819
:101770009001002005490C31086001200549C1F89D
:10178000B00108BD000C01400008014098812142D1
:10179000000021420080214210B50446022223218C
:1017A000204600F0D5FC05231E4A2A21204600F0E1
:1017B00091FC05231B4A3021204600F08BFC3F2280
:1017C0002121204600F0C4FC01222221204600F005
:1017D000BFFC1A222521204600F0BAFC2422262133
:1017E000204600F0B5FC0F222021204600F0B0FC7E
:1017F0000A223121204600F0ABFC01223D21204687
:1018000000F0A6FC00223C21204600F0A1FC702242
:101810002721204600F09CFCFF22E221204600F018
:1018200097FC10BD753A000810B50446022223212A
:10183000204600F08DFC05231E4A2A21204600F098
:1018400049FC05231B4A3021204600F043FC3F227F
:101850002121204600F07CFC01222221204600F0BC
:1018600077FC12222521204600F072FC042226215A
:10187000204600F06DFC0F222021204600F068FC7D
:101880000A223121204600F063FC01223D2120463E
:1018900000F05EFC00223C21204600F059FC702242
:1018A0002721204600F054FCFF22E221204600F0D0
:1018B0004FFC10BD663A000810B5044602222321F1
:1018C000204600F045FC05231E4A2A21204600F050
:1018D00001FC05231B4A3021204600F0FBFB30228F
:1018E0002121204600F034FC01222221204600F074
:1018F0002FFC12222521204600F02AFC212226213D
:10190000204600F025FC0F222021204600F020FC7C
:101910000A223121204600F01BFC00223D212046F6
:1019200000F016FC01223C21204600F011FC702240
:101930002721204600F00CFCFF22E221204600F087
:1019400007FC10BD573A000810B5044601222321B8
:10195000204600F0FDFB05231E4A2A21204600F008
:10196000B9FB05231B4A3021204600F0B3FB30228F
:101970002121204600F0ECFB01222221204600F02C
:10198000E7FB19222521204600F0E2FB0422262154
:10199000204600F0DDFB0F222021204600F0D8FB7E
:1019A00006223121204600F0D3FB01223D212046B2
:1019B00000F0CEFB00223C21204600F0C9FB702243
:1019C0002721204600F0C4FBFF22E221204600F040
:1019D000BFFB10BD843A000810B504461CB90020B6
:1019E0002749086003E0002025490C3108600122E6
:1019F0002321204600F0ACFB0323224A2A21204663
:101A000000F068FB0323204A3021204600F062FBEF
:101A100001222121204600F09BFB012222212046A9
:101A200000F096FB2A222521204600F091FB04229B
:101A30002621204600F08CFB0F222021204600F0BA
:101A400087FB06223D21204600F082FB01223C213B
:101A5000204600F07DFB70222721204600F078FB15
:101A6000FF22E221204600F073FB1CB9012004494B
:101A7000086003E0012002490C31086010BD00003D
:101A8000988121424D3A0008483A000870B5044652
:101A90000D461CB900202649086003E000202449B7
:101AA0000C3108600C2D37D2DFE805F0060A0E1263
:101AB000161A1E22262A2E322046FFF7FDFE2BE0A4
:101AC000204600F09FF927E0204600F02BFA23E0A3
:101AD0002046FFF7A9FE1FE0204600F003F91BE0B7
:101AE000204600F06FF817E02046FFF755FE13E0A0
:101AF000204600F0AFF80FE0204600F0CBF90BE0F5
:101B00002046FFF721FF07E0204600F013F803E02E
:101B1000204600F02FF900BF00BF1CB90120044986
:101B2000086003E0012002490C31086070BD00002C
:101B30009881214210B5044602222321204600F05C
:101B400007FB04231E4A2A21204600F0C3FA04237F
:101B50001B4A3021204600F0BDFA302221212046C8
:101B600000F0F6FA01222221204600F0F1FA2022AC
:101B70002521204600F0ECFA20222621204600F004
:101B8000E7FA0F222021204600F0E2FA0822312154
:101B9000204600F0DDFA01223D21204600F0D8FA6F
:101BA00000223C21204600F0D3FA70222721204653
:101BB00000F0CEFAFF22E221204600F0C9FA10BD63
:101BC000893A000810B5044602222321204600F07D
:101BD000BFFA05231E4A2A21204600F07BFA05237E
:101BE0001B4A3021204600F075FA30222121204680
:101BF00000F0AEFA01222221204600F0A9FA1222BA
:101C00002521204600F0A4FA24222621204600F0B7
:101C10009FFA0F222021204600F09AFA0A22312151
:101C2000204600F095FA01223D21204600F090FA6E
:101C300000223C21204600F08BFA7022272120460A
:101C400000F086FAFF22E221204600F081FA10BD62
:101C5000703A000810B5044601222321204600F006
:101C600077FA05231E4A2A21204600F033FA05237D
:101C70001B4A3021204600F02DFA30222121204637
:101C800000F066FA01222221204600F061FA1022BB
:101C90002521204600F05CFA04222621204600F08F
:101CA00057FA0F222021204600F052FA0622312155
:101CB000204600F04DFA01223D21204600F048FA6E
:101CC00000223C21204600F043FA702227212046C2
:101CD00000F03EFAFF22E221204600F039FA10BD62
:101CE0007A3A000810B5044602222321204600F06B
:101CF0002FFA05231E4A2A21204600F0EBF905237E
:101D00001B4A3021204600F0E5F9302221212046EF
:101D100000F01EFA01222221204600F019FA1222B8
:101D20002521204600F014FA24222621204600F026
:101D30000FFA0F222021204600F00AFA0822312152
:101D4000204600F005FA01223D21204600F000FA6D
:101D500000223C21204600F0FBF97022272120467A
:101D600000F0F6F9FF22E221204600F0F1F910BD63
:101D70006B3A000810B5044602222321204600F0E9
:101D8000E7F904231E4A2A21204600F0A3F9042380
:101D90001B4A3021204600F09DF9302221212046A7
:101DA00000F0D6F901222221204600F0D1F91C22B0
:101DB0002521204600F0CCF924222621204600F0DF
:101DC000C7F90F222021204600F0C2F90822312154
:101DD000204600F0BDF901223D21204600F0B8F96F
:101DE00000223C21204600F0B3F970222721204632
:101DF00000F0AEF9FF22E221204600F0A9F910BD63
:101E00008E3A000810B5044603222321204600F034
:101E10009FF905231E4A2A21204600F05BF905237D
:101E20001B4A3021204600F055F93F22212120464F
:101E300000F08EF93F222221204600F089F9282265
:101E40002521204600F084F904222621204600F0B6
:101E50007FF90B222021204600F07AF90A22312155
:101E6000204600F075F901223D21204600F070F96E
:101E700000223C21204600F06BF9702227212046E9
:101E800000F066F9FF22E221204600F061F910BD62
:101E90005C3A000810B5044601222321204600F0D8
:101EA00057F903231E4A2A21204600F013F9032381
:101EB0001B4A3021204600F00DF930222121204616
:101EC00000F046F901222221204600F041F92A22A1
:101ED0002521204600F03CF904222621204600F06E
:101EE00037F90F222021204600F032F90722312154
:101EF000204600F02DF900223D21204600F028F96F
:101F000001223C21204600F023F97022272120469F
:101F100000F01EF9FF22E221204600F019F910BD61
:101F20007F3A000810B5044603222321204600F022
:101F30000FF905231E4A2A21204600F0CBF805237D
:101F40001B4A3021204600F0C5F8302221212046CE
:101F500000F0FEF801222221204600F0F9F81022BC
:101F60002521204600F0F4F804222621204600F026
:101F7000EFF80F222021204600F0EAF80A22312152
:101F8000204600F0E5F801223D21204600F0E0F86F
:101F900000223C21204600F0DBF870222721204659
:101FA00000F0D6F8FF22E221204600F0D1F810BD63
:101FB000613A00082DE9F0478046894615461E46DD
:101FC000B8F1000F16D10020174908604946404675
:101FD00000F0F4FB0746002406E0FF21404600F035
:101FE000EDFB2855601CC4B2B442F6DB01200E495B
:101FF000086015E000200D4908604946404600F0A1
:10200000DDFB0746002406E0FF21404600F0D6FB3A
:102010002855601CC4B2B442F6DB012003490860B5
:102020003846BDE8F087000090012142B08121428E
:1020300070B505460E4685B9002011490860314645
:10204000284600F0BBFBFF21284600F0B7FB044602
:1020500001200C49C1F890010FE000200A490860F6
:102060003146284600F0AAFBFF21284600F0A6FBD7
:10207000044601200549C1F8B001204670BD0000AA
:102080009001214200002142B08121420080214282
:1020900070B506460D461021304600F0E3FB0721DF
:1020A0003046FFF7C5FF044622462721304600F0A0
:1020B0004FF804F0400050B10A232A46612130460F
:1020C000FFF778FFFF22E221304600F041F820467A
:1020D00070BD00002DE9F0478046894615461E4632
:1020E000B8F1000F16D10020174908604946404654
:1020F00000F064FB0746002406E015F8011B40468B
:1021000000F05CFB601CC4B2B442F6DB01200E4957
:10211000086015E000200D4908604946404600F07F
:102120004DFB0746002406E015F8011B404600F071
:1021300045FB601CC4B2B442F6DB012003490860D1
:102140003846BDE8F087000090012142B08121426D
:102150002DE9F04104460E46154684B90020114988
:1021600008603146204600F029FB074629462046F4
:1021700000F024FB01200C49C1F890010FE0002081
:102180000A4908603146204600F018FB07462946F8
:10219000204600F013FB01200549C1F8B001384684
:1021A000BDE8F0819001214200002142B08121422E
:1021B0000080214208B54FF4C06000F071F826207D
:1021C0008DF8000001208DF8010002208DF802003A
:1021D00001208DF80300684600F02AF827208DF8CA
:1021E000000001208DF801008DF802008DF8030039
:1021F000684600F01DF825208DF8000000208DF8BD
:10220000010001208DF802008DF80300684600F0FF
:102210000FF81D208DF8000000208DF801008DF8CA
:10222000020001208DF80300684600F001F808BDA7
:1022300070B5002100230F22C47804B3154C246824
:1022400004F4E064C4F5E064210AC1F10403CA4067
:10225000447804FA03F184781440214309010E4CB8
:102260000678A155047804F01F050124AC400578D8
:102270006D11AD0005F1E025C5F8004109E00478D5
:1022800004F01F050124AC40044D0678761145F892
:10229000264070BD0CED00E000E400E080E100E0CD
:1022A00002490143024A1160704700000000FA052C
:1022B0000CED00E07047000029B1064AD2690243E4
:1022C000044BDA6104E0034AD2698243014BDA61CC
:1022D000704700000010024029B1064A926902438B
:1022E000044B9A6104E0034A92698243014B9A616C
:1022F000704700000010024010B500F033F84FF4B2
:10230000803000F0F1F800F04DF90446012C1ED1A8
:10231000002000F0DDF8002000F018F9A00200F025
:1023200009F94FF4E011200400F022F9012000F037
:1023300019F900BF392000F0A5F80028FAD00220D2
:1023400000F024F900BF00F0BBF80828FBD1012100
:1023500044F20D00FFF7C0FF01210220FFF7ACFFA0
:1023600010BD00000F48006840F001000D490860F2
:10237000084640680C4908400A4948600846006819
:102380000A490840074908600846006820F4802090
:1023900008600846406820F4FE0048604FF41F00C3
:1023A00088607047001002400000FFF8FFFFF6FE53
:1023B00030B500210022002400232D4D6D6805F06A
:1023C0000C0121B1042905D0082923D105E0294DAC
:1023D000056022E0274D05601FE0254D6D6805F47E
:1023E0007012234D6D6805F48034022505EB92428E
:1023F0001CB9214D554305600BE01D4D6D6805F47A
:1024000000351DB11C4D5543056002E0194D554383
:10241000056002E0174D056000BF00BF144D6D68F8
:1024200005F0F0010909154D6B5C0568DD4045605C
:102430000F4D6D6805F4E061090A104D6B5C45684D
:10244000DD4085600A4D6D6805F46051C90A0B4D89
:102450006B5C4568DD40C560054D6D6805F4404125
:10246000890B074D6B5CC568B5FBF3F5056130BDA5
:102470000010024000127A0000093D009400002084
:10248000A400002010B501460022002300204A11BC
:10249000012A02D1094C236806E0022A02D1074C26
:1024A000236A01E0054C636A01F01F020124944095
:1024B0001C400CB1012000E0002010BD00100240C3
:1024C0000248406800F00C00704700000010024015
:1024D00001460020034A506820F0F0000843506095
:1024E00070470000001002401149096821F4803152
:1024F0000F4A11601146096821F480211160B0F57E
:10250000803F03D0B0F5802F0ED106E0084909685E
:1025100041F48031064A116007E00549096841F439
:10252000A021034A116000E000BF00BF7047000017
:102530000010024001460020034A506820F4E06089
:102540000843506070470000001002400146002020
:10255000034A506820F4605040EAC1005060704760
:102560000010024001490866704700000000424226
:1025700002460020044B586820F47C1042EA010314
:102580001843014B5860704700100240014600207C
:10259000034A506820F00300084350607047000071
:1025A0000010024038B5002000900024002500BF34
:1025B0003120FFF767FF05460098401C0090009807
:1025C000B0F5A06F01D0002DF2D03120FFF75AFFF7
:1025D00008B1012400E00024204638BD10B586B0C3
:1025E0000024142101A8FDF7D8FD0A2201A90848FA
:1025F00000F012F800BF07E001A810F81400054A27
:1026000002F81400601CC4B20A2CF5DB06B010BD41
:10261000000003084C05002070B504460D46164620
:10262000002300BF07E02046FEF76CFE25F81300EC
:10263000A41C581CC3B2B342F5DB70BD00B587B013
:10264000012141F20500FFF747FEE020ADF8180038
:1026500018208DF81B0003208DF81A0006A91648D3
:10266000FEF7C1FDE0211448FEF74AFE0020ADF858
:1026700004004FF48270ADF806000020ADF80800A9
:10268000ADF80A00ADF80C004FF40070ADF80E0084
:102690001820ADF810000020ADF812000720ADF8AA
:1026A000140001A9054800F06BF80121034800F06F
:1026B0004DF807B000BD00000008014000300140A7
:1026C00000B587B001218803FFF7F6FD012109203D
:1026D000FFF702FE4FF46040ADF8180018208DF8A7
:1026E0001B0003208DF81A0006A91648FEF77BFD93
:1026F0004FF460411348FEF703FE0020ADF80400DC
:102700004FF48270ADF806000020ADF80800ADF877
:102710000A00ADF80C004FF40070ADF80E00182060
:10272000ADF810000020ADF812000720ADF814003D
:1027300001A9054800F024F80121034800F006F83B
:1027400007B000BD000C01400038004021B10288F4
:1027500042F04002028004E002884FF6BF731A4044
:10276000028070470246002013890B400BB1012004
:1027700000E00020704701468889704781817047DA
:1027800010B50022028802F441520B884C88234382
:102790008C882343CC8823430C8923434C892343CF
:1027A0008C892343CC8923431A430280838B4FF2C5
:1027B000FF74234083830B8A038210BD2DE9F0410F
:1027C00006460F4626BB06E0601CC4B2C82C02DBDE
:1027D0000020BDE8F08102212048FFF7C3FF002858
:1027E000F2D039461D48FFF7C9FF002405E0601C00
:1027F000C4B2C82C01DB0020EBE701211748FFF72A
:10280000B1FF0028F3D01548FFF7B5FFC5B222E0AD
:1028100005E0601CC4B2C82C01DB0020D9E702210E
:102820000F48FFF79FFF0028F3D039460C48FFF709
:10283000A5FF002405E0601CC4B2C82C01DB002009
:10284000C7E701210648FFF78DFF0028F3D00448B1
:10285000FFF791FFC5B22846BBE7000000300140FA
:102860000038004070B505460C467DB90F48008819
:102870004FF6C77108400D4908800846008820437C
:10288000088001210A48FFF761FF0EE00848008830
:102890004FF6C77108400649088008460088204363
:1028A000088001210248FFF751FF70BD0030014050
:1028B00000380040704770B504460D462946204652
:1028C000FEF752FC70BD000010B586B00024142144
:1028D00001A8FDF762FC00BF07E00B4830F81400C8
:1028E00001A921F81400601CC4B20A2CF5DB0748CA
:1028F00000F008F90A2201A9044800F009F800F0E4
:1029000082FC06B010BD000038050020000003085E
:102910002DE9F04105460F461646002400BF07E0AA
:1029200037F814102846FFF7C6FFAD1C601CC4B270
:10293000B442F5DBBDE8F08170B504460D46034AAC
:102940002946204600F028F870BD000000380140FC
:1029500010B504460249204600F00EF810BD0000F4
:102960000044004010B504460249204600F02DF80E
:1029700010BD00000044004070B504460D4600BF85
:102980008021284600F06CFB0028F9D0214628461B
:1029900000F033FC012070BD2DE9F04104460D46E6
:1029A000164614B90120BDE8F0810AE014F8017B55
:1029B00031463846FFF7E0FF08B90020F3E7681E0C
:1029C00085B2002DF2D10120EDE770B504460E4628
:1029D0000CB9012070BD11E014F8015B0A2D06D17D
:1029E00031460D20FFF7C8FF08B90020F2E7314655
:1029F0002846FFF7C1FF08B90020EBE72078002840
:102A0000EAD10120E6E70178032903DA0178891C7D
:102A1000017002E00178891E0170704710B500F066
:102A200001F810BD0CB500200190009033480068FB
:102A300040F480303149086000BF3048006800F43D
:102A4000003000900198401C0190009818B901983E
:102A5000B0F5A06FF1D12948006800F4003010B142
:102A60000120009001E0002000900098012843D14F
:102A70002348006840F010002149086008460068BB
:102A800020F0030008600846006840F0020008607B
:102A90001A48406819494860084640684860084636
:102AA000406840F4806048600846406820F47C102C
:102AB00048600846406840F4E810486008460068EE
:102AC00040F08070086000BF0C48006800F00070A3
:102AD0000028F9D00948406820F003000749486001
:102AE0000846406840F00200486000BF0348406864
:102AF00000F00C000828F9D10CBD000000100240C5
:102B00000020024010B50446FEF74EFB2046FEF7BB
:102B1000E1FA10BD7047000010B51348006840F09E
:102B200001001149086008464068104908400E49F4
:102B30004860084600680E4908400B49086008468E
:102B4000006820F4802008600846406820F4FE00F9
:102B500048604FF41F008860FFF760FF4FF000608F
:102B60000449086010BD0000001002400000FFF89A
:102B7000FFFFF6FE08ED00E010B50121204800F04F
:102B80007EF800283AD001211D4800F069F81D4860
:102B90000088401C1B4908801B480088401C1A49BB
:102BA00008801A480088401C184908801848007896
:102BB000C0B14FF400711748FEF7A2FB1648008819
:102BC000401C1549088008460088B0F5C87F09DB1D
:102BD0004FF400710F48FEF791FB00200E4908806A
:102BE0000B4908700948008841F28831884202D1B7
:102BF00000200649088001200849087010BD000027
:102C000000040040200000203200002022000020AC
:102C10002500002000100140260000202400002094
:102C20003EB505460C4601210220FFF745FBADF8F5
:102C30000450ADF800400020ADF80600ADF80200E9
:102C40006946064800F036F801221146034800F0B4
:102C500027F80121014800F006F83EBD00040040BD
:102C6000CA430282704721B1028842F00102028009
:102C700004E002884FF6FE731A400280704730B5B8
:102C80000246002000230024158A05EA01039589E5
:102C900005EA010413B10CB1012000E0002030BDB1
:102CA0001AB183890B43838102E083898B4383813B
:102CB00070470000002202881D4B98420ED01D4B29
:102CC00098420BD0B0F1804F08D01B4B984205D0F2
:102CD0001A4B984202D01A4B984204D14FF68F7388
:102CE0001A404B881A43174B984207D0164B98420C
:102CF00004D04FF6FF431A40CB881A4302808B88DA
:102D000083850B8803850A4B98420BD0094B984268
:102D100008D00E4B984205D00D4B984202D00D4B77
:102D2000984201D10B7A0386012383827047000009
:102D3000002C014000340140000400400008004025
:102D4000000C004000100040001400400040014012
:102D5000004401400048014010B540F2255112489E
:102D600000F08BF988B140F225510F4800F0CFF800
:102D70000D4800F03DFAC4B20C480D49097844549E
:102D80000B480078401C0A4908700821064800F0EA
:102D900067F9012806D10821034800F0AFF802487E
:102DA00000F026FA10BD000000380140100100209C
:102DB0000300002010B540F22551124800F05DF9E3
:102DC00088B140F225510F4800F0A1F80D4800F0FD
:102DD0000FFAC4B20C480D49097844540B480078E6
:102DE000401C0A4908700821064800F039F90128FA
:102DF00006D10821034800F081F8024800F0F8F9F4
:102E000010BD000000440040F804002085000020B0
:102E100010B586B0044601210520FFF75DFA0121B7
:102E20004804FFF749FA0420ADF8140003208DF898
:102E3000160018208DF8170005A91548FEF7D3F9DC
:102E40000820ADF8140004208DF8170005A91048DB
:102E5000FEF7C9F901940020ADF80800ADF80A00AA
:102E6000ADF80C00ADF810000C20ADF80E0001A973
:102E7000084800F051F9012240F22551054800F0C0
:102E800026F90121034800F051F806B010BD0000FA
:102E9000000801400044004010B540F2255114489C
:102EA00000F0EBF8B0B140F22551114800F02FF8D6
:102EB0000F4800F09DF9C4B20E480F4909784454F8
:102EC0000D480078401C0C4908700846007800F056
:102ED0000F0008700821064800F0C2F8012806D14A
:102EE0000821034800F00AF8014800F081F910BDFC
:102EF00000480040D80100200900002001F40072C1
:102F0000B2F5007F00D100BFCA430280704710B500
:102F10000022002340F66A14A14200D100BF0A1229
:102F200001249440A3B2DC43048010BD21B1828906
:102F300042F40052828104E082894DF6FF731A4008
:102F40008281704700B585B0012144F20400FFF78B
:102F5000C3F94FF40070ADF8000003208DF80200B3
:102F600018208DF8030069463948FEF73CF94FF404
:102F70008060ADF8000004208DF8030069463448F5
:102F8000FEF731F94FF4164001900020ADF808002B
:102F9000ADF80A00ADF80C00ADF810000C20ADF84B
:102FA0000E0001A92B4800F0B7F8012240F225518C
:102FB000284800F08CF801212648FFF7B7FF0121CF
:102FC0008804FFF779F901210820FFF785F94FF40C
:102FD0008060ADF8000003208DF8020018208DF805
:102FE000030069461C48FEF7FEF84FF40060ADF898
:102FF000000004208DF8030069461748FEF7F3F837
:103000004FF4965001900020ADF80800ADF80A008A
:10301000ADF80C00ADF810000C20ADF80E0001A9C1
:103020000E4800F079F801A90C4800F075F801226B
:1030300040F22551094800F04AF801210748FFF7FE
:1030400075FF40210348FFF759FF05B000BD0000A0
:103050000008014000380140000C014000480040D9
:1030600002460020B1F5007F00D100BF13880B405D
:103070000BB1012000E00020704770B5024600242B
:1030800000230025002040F66A16B14200D100BF9F
:10309000C1F3421501F01F03012606FA03F3012DC7
:1030A00002D19689334006E0022D02D1168A3340C0
:1030B00001E0968A33400C12012606FA04F41688C1
:1030C000344013B10CB1012000E0002070BDF0B518
:1030D0000346002400260025002040F66A17B94266
:1030E00000D100BF1846C1F3421401F01F060127AA
:1030F00007FA06F5012C01D10C3004E0022C01D1B5
:10310000103000E014301AB107682F43076002E066
:103110000768AF430760F0BD2DE9F04786B005466C
:103120000E460024A24600BFA1460027B08900B188
:1031300000BF2F462C8A4CF6FF700440F0880443F1
:103140002C82AC894EF6F3100440B08831890843D4
:10315000718908430443AC81AC8A4FF6FF400440B8
:10316000B0890443AC8201A8FFF722F91F488742C7
:1031700002D1DDF810A001E0DDF80CA0A88900F470
:10318000004040B10AEBCA0000EB0A103168490068
:10319000B0FBF1F807E00AEBCA0000EB0A10316857
:1031A0008900B0FBF1F86420B8FBF0F004012009BD
:1031B000642101FB1089A88900F4004040B132204D
:1031C00000EBC900B0FBF1F000F00700044308E099
:1031D000322000EB09106421B0FBF1F000F00F0089
:1031E00004432C8106B0BDE8F087000000380140A0
:1031F00001468888C0F308007047C1F30802828046
:10320000704700BFFEE710B5FDF7A4FF10BD00003A
:10321000014A024900F013B8DD330008A80000207D
:1032200002E008C8121F08C1002AFAD1704770478F
:10323000002001E001C1121F002AFBD170472DE9D7
:10324000F04116460F460446002503E03946B047D4
:10325000641C6D1C20780028F8D12846BDE8F08158
:1032600070B505460C4605F1B001C8B207490968BA
:103270008847102101EB241004490968884704F0AD
:103280000F0002490968884770BD00008C000020CB
:1032900010B54FF480511E48FEF732F804211C4847
:1032A000FEF72CF84FF480611948FEF729F8002446
:1032B00021E04FF400611648FEF720F81548007829
:1032C00000F0800028B94FF480511148FEF716F83D
:1032D00004E04FF480510E48FEF712F80D480078D4
:1032E0004006000E0B4908704FF400610848FEF7D5
:1032F00007F8601CC4B2082CDBDB04210448FDF78E
:10330000FFFF4FF480510248FDF7FAFF10BD0000A7
:10331000001001408800002070B5044600BF4FF443
:1033200080511B48FDF7ECFF04211948FDF7E6FF2B
:103330004FF480611648FDF7E1FF00251BE04FF4D4
:1033400000611348FDF7DAFF04F0800028B94FF45C
:1033500080510F48FDF7D2FF04E04FF480510C4834
:10336000FDF7CEFF6006040E4FF400610848FDF73C
:10337000C7FF681CC5B2082DE1DB04210448FDF736
:10338000BFFF4FF480510248FDF7BAFF70BD000047
:1033900000100140014605E0122001E0421E90B2FB
:1033A0000028FBDC0A00A1F1010399B2F4D17047B7
:1033B00010B502460BE0C82007E0122101E04B1EC9
:1033C00099B20029FBDC431E98B20028F5DC1300FB
:1033D000A2F10104A2B2EED110BD000070B5044606
:1033E0000D46E0B20549088000BF40210348001F98
:1033F000FFF736FE0028F8D0204670BD04380140A3
:1034000008B50120ADF8000010208DF8030003205E
:103410008DF8020069461A48FDF7E5FE0420ADF874
:10342000000069461648FDF7DEFE0820ADF80000F2
:1034300069461348FDF7D7FE4FF48060ADF80000F1
:1034400069460F48FDF7CFFE4FF40060ADF800006D
:1034500069460B48FDF7C7FE4FF48050ADF80000F9
:1034600069460748FDF7BFFE01210548FDF748FF03
:103470001821002000F046FA00F0DCF908BD000039
:103480000010014008B501211020FEF725FF0120A2
:10349000ADF8000010208DF8030003208DF8020025
:1034A00069460D48FDF79FFE01210B48FDF728FFF7
:1034B0004FF40070ADF8000010208DF803000320D9
:1034C0008DF8020069460448FDF78DFE4FF4007147
:1034D0000148FDF713FF08BD00100140FEF70CFF87
:1034E000FEF768FE40F271210420FEF77FF8FEF738
:1034F00079F841F61F410920FFF792FBFFF7C2FF61
:10350000FFF77EFFFCF766FEFFF71CFD4FF4E1308E
:10351000FFF77EFCFEF7C6F8FEF764F802E072A043
:10352000FFF776FE0120FEF791F80028F7D1FDF7AE
:10353000BDFCFEF757F870480068C0436F49C1F8FA
:103540008001C820FFF734FF6C48D0F88001C043E9
:103550006A49C1F88001062169A0FDF748FD6AA00B
:10356000FFF700FAFEF73EF868A0FFF751FE0120D2
:10357000FEF732FAFFF732F86B4800786B490870B3
:10358000084600780C2813D2DFE800F00613202D3F
:103590003A4754616E7B889565A0FFF739FE01209C
:1035A00000F06EF9072365A20121084600F02CFA0D
:1035B0008EE064A0FFF72CFE012000F061F90523E6
:1035C00063A20121084600F01FFA81E062A0FFF724
:1035D0001FFE012000F054F9062362A201210846D3
:1035E00000F012FA74E061A0FFF712FE012000F073
:1035F00047F9072360A20121084600F005FA67E0B9
:103600005FA0FFF705FE012000F03AF907235FA253
:103610000121084600F0F8F95AE05EA0FFF7F8FD36
:10362000012000F02DF909235EA20121084600F0D7
:10363000EBF94DE05EA0FFF7EBFD012000F020F973
:1036400005235EA20121084600F0DEF940E05DA0FE
:10365000FFF7DEFD012000F013F906235CA2012133
:10366000084600F0D1F933E05BA0FFF7D1FD01205F
:1036700000F006F904235BA20121084600F0C4F91A
:1036800026E05AA0FFF7C4FD012000F0F9F80D2351
:1036900059A20121084600F0B7F919E05AA0FFF736
:1036A000B7FD012000F0ECF80B235AA201210846D7
:1036B00000F0AAF90CE05AA0FFF7AAFD012000F0E3
:1036C000DFF802235AA20121084600F09DF900BF4D
:1036D00000BF3220FFF76CFE05E0FCF7D9FDFDF7D7
:1036E00035F8FDF7DDF8F8E754686520322E3447E9
:1036F000204572726F722100800122420000224236
:1037000031323334353600000A0000000A5043B627
:10371000D4C2EBC8EDBCFECDA8D3C3B0E6B1BE5653
:10372000312E370A000000004C0500202A0000203E
:10373000BDADCEF7D0ADD2E90D0A00004A49414EE9
:1037400047584900CCECB2A8D0ADD2E90D0A000030
:1037500054454C504F000000D4C6C4CFD0ADD2E980
:103760000D0A000059554E4E414E0000B9F3D6DD0A
:10377000D0ADD2E90D0A00004755495A484F5500CF
:10378000CBC4B4A8D0ADD2E90D0A000053494348D8
:1037900055414E00C4DAC3C9B9C5D0ADD2E90D0A4E
:1037A000000000004E45494D454E4747550000007A
:1037B000B0B2BBD5D0ADD2E90D0A0000414E48559C
:1037C00049000000C9BDCEF7D0ADD2E90D0A000016
:1037D0005348414E5849000056434F4DB2E2CAD4B7
:1037E0000D0A000056434F4D00000000C1C9C4FE41
:1037F000B5E7D0C50D0A00004C49414F4E494E4730
:103800002E4449414E000000C1C9C4FED2C6B6AF25
:103810000D0A00004C49414F4E494E472E59490070
:103820005470D7A8D3C3D0ADD2E90D0A0000000070
:103830005450000070B5002411E000200D490870BC
:1038400000212046FFF70CFD002504E00A4800682F
:103850008047681CC5B2852DF8DB601CC4B2082CFB
:10386000EBDBAF200549096888472F200349096829
:10387000884770BD88000020900000208C00002048
:1038800031B56846FFF7BFF89DF80000401EC0B292
:103890000090042800DB38BD9DF800004006000EB3
:1038A0000090002525E000219DF80000FFF7D8FCDE
:1038B000002012490870002404E011480068804785
:1038C000601CC4B2802CF8DB9DF80010491CC8B203
:1038D0000021FFF7C5FC002008490870002404E01F
:1038E000074800688047601CC4B2802CF8DB681C65
:1038F000C5B2022DD7DB00BFCDE700008800002055
:103900009000002070B504460D4605480549086042
:103910000548064908602946204600F009F870BDB0
:10392000193300088C00002091320008900000201C
:1039300070B505460C4605B34FF480513048FDF78D
:10394000DFFC0120FFF726FD08212D48FDF7D8FCFC
:1039500004212B48FDF7D2FC0520FFF729FD0821A3
:103960002748FDF7CBFC1E20FFF722FD0821244845
:10397000FDF7C6FC1320FFF71BFD04212048FDF7CF
:10398000BDFC4FF480511E48FDF7BAFC08211C48CD
:10399000FDF7B6FCA2201B4909688847A0201949F9
:1039A00009688847C820174909688847A62015492B
:1039B000096888472F201349096888470220FFF7C4
:1039C000E9FCF8200F490968884701200D4909687A
:1039D000884724200B490968884724248120094905
:1039E000096888472046074909688847AF20054984
:1039F00009688847602003490968884770BD00004E
:103A0000001001408C0000202DE9FF4781460E4642
:103A100017461D46002D01DCBDE8FF8700240FE09E
:103A200017F80480601C84B269464046FDF76EFCBE
:103A300008236A4631464846FDF7F4FA701CC6B2C0
:103A4000AC42EDDB00BFE7E7344310100134431014
:103A5000100133200D547933200D54793443101064
:103A60000101101043343223ABBA013412BBAA0156
:103A700034128675014656431000346E46100134E8
:103A800043101001862C95010136E4A7BC014218B1
:103A9000BAE801F8FC04C424FCF800070F09080880
:103AA0000F0700001018FCFC0000000008080F0FB2
:103AB000080800080C84C4643C18000E0F090808AC
:103AC0000C0C00080C444444FCB800040C08080822
:103AD0000F0700C0E0B098FCFC8000000000080F59
:103AE0000F08007C7C4444C4C48400040C0808080B
:103AF0000F0700F0F84C4444C08000070F08080886
:103B00000F07000C0C0484C47C3C0000000F0F0065
:103B1000000000B8FC444444FCB800070F08080843
:103B20000F0700387C444444FCF800000808080CE7
:103B3000070300E0F0988C98F0E0000F0F00000001
:103B40000F0F0004FCFC4444FCB800080F0F0808E9
:103B50000F0700F0F80C04040C180003070C080809
:103B60000C060004FCFC040CF8F000080F0F080C15
:103B700007030004FCFC44E40C1C00080F0F0808B9
:103B80000C0E0004FCFC44E40C1C00080F0F0800A1
:103B9000000000F0F80C84848C980003070C0808DF
:103BA000070F00FCFC404040FCFC000F0F00000031
:103BB0000F0F00000004FCFC0400000000080F0FC1
:103BC00008000000000004FCFC0400070F08080FB8
:103BD00007000004FCFCC0F03C0C00080F0F0001C3
:103BE0000F0E0004FCFC0400000000080F0F080882
:103BF0000C0E00FCFC387038FCFC000F0F000000BD
:103C00000F0F00FCFC3870E0FCFC000F0F00000000
:103C10000F0F00F0F80C040CF8F00003070C080C70
:103C200007030004FCFC44447C3800080F0F080024
:103C3000000000F8FC040404FCF800070F080E3C28
:103C40003F270004FCFC44C4FC3800080F0F0000B0
:103C50000F0F00183C6444C49C1800060E080808A6
:103C60000F0700001C0CFCFC0C1C000000080F0FD0
:103C7000080000FCFC000000FCFC00070F0808081E
:103C80000F0700FCFC000000FCFC000103060C0612
:103C9000030100FCFC008000FCFC00030F0E030E7F
:103CA0000F03000C3CF0C0F03C0C000C0F030003B1
:103CB0000F0C00003C7CC0C07C3C000000080F0FD3
:103CC0000800001C0C84C4643C1C000E0F0908088A
:103CD0000C0E0000000000000000000000000C0CB2
:103CE0000000000000003030000000000000060668
:103CF00000000000143D000800000020AC0000009F
:103D000020320008C03D0008AC000020545F0000D5
:103D10003032000800000000000000000000000039
:103D2000D1D1E0D000000000D2D20000000000009D
:103D30000000000000000000000000000000000083
:103D40000000000000000000000000000000000073
:103D50000000000000003132333435363738393155
:103D600032333435363738390000000000000000A7
:103D70000000000000003132333435363738393135
:103D80003233343536373839000000000000000087
:103D90000000000000000000000000000000000023
:103DA0000000000000000000000000000102030409
:103DB00001020304060708090204060800000000C7
:0400000508000131BD
:00000001FF
